:020000040800F2
:100000009006002031020008C9230008712300086F
:10001000C52300088D080008C52C0008000000005A
:10002000000000000000000000000000A5250008FE
:100030009108000800000000CB230008A725000855
:100040005502000855020008550200085502000834
:100050005502000855020008550200085502000824
:100060005502000855020008550200085502000814
:100070005502000855020008550200085502000804
:1000800055020008550200085502000855020008F4
:10009000550200085502000855020008CD08000866
:1000A00055020008550200085502000855020008D4
:1000B00055020008550200085502000855020008C4
:1000C00055020008550200085502000855020008B4
:1000D00055020008752C000855020008550200085A
:1000E000950800085502000855020008550200084E
:1000F0005502000855020008550200085502000884
:100100005502000855020008550200085502000873
:100110005502000855020008550200085502000863
:100120005502000855020008550200085502000853
:100130005502000855020008550200085502000843
:100140005502000855020008550200085502000833
:100150005502000855020008550200085502000823
:100160005502000855020008550200085502000813
:100170005502000855020008550200080000000062
:10018000550200085502000800F002F800F041F89E
:100190000AA090E8000C82448344AAF10107DA45E2
:1001A00001D100F036F8AFF2090EBAE80F0013F0F3
:1001B000010F18BFFB1A43F001031847682D000018
:1001C000882D0000103A24BF78C878C1FAD85207A9
:1001D00024BF30C830C144BF04680C6070470000C1
:1001E0000023002400250026103A28BF78C1FBD840
:1001F000520728BF30C148BF0B607047642900F028
:10020000F580002070471FB502F07AFE1FBD10B5C3
:1002100010BD00F0FBF91146FFF7F5FF02F0B4FD49
:1002200000F019FA03B4FFF7F2FF03BC02F068FD17
:100230000C48016841F4700101600B4880470B488D
:100240000047FEE7FEE7FEE7FEE7FEE7FEE7FEE724
:10025000FEE7FEE7FEE7000005480649044A064BB4
:100260007047000088ED00E0B12500088901000812
:10027000900200209006002090020020704753EA70
:10028000020C00F069802DE9F04B4FF00006002BC6
:100290001FBFB3FA83F503FA05F424FA05F65E40AE
:1002A00012BF1643B2FA82F502FA05F4C5F1200531
:1002B0001EBF22FA05FC44EA0C04203556EA044C21
:1002C0004FEA144418BF641C4FF000084FF00009B7
:1002D000904271EB030C39D3002919BFB1FA81F7B1
:1002E00001FA07F6B0FA80F700FA07F6C7F120071F
:1002F0001EBF20FA07FC46EA0C062037B6FBF4FCCA
:10030000A7EB0507103F07F01F0BCBF120060CFAF7
:100310000BFB2CFA06F644BFB3460026202FA4BFE1
:100320005E464FF0000B5BEA060C08BF4FF0010B76
:1003300019EB0B09ABFB027C48EB0608C01B06FB64
:1003400002CC0BFB03CC71EB0C01C1E70B46024660
:1003500041464846BDE8F08B13B54FF000004FF022
:100360000001AFF30080BDE81C4070470FB40449A2
:1003700010B503AA029800F01BF910BC5DF814FB3D
:100380000C0000202DE9F0410E46044600202062BA
:100390002046E168884730B3252805D0D4E90121FB
:1003A0009047206A401CF2E7E16820460027884712
:1003B000050018D0A5F14100192802D820354FF4C6
:1003C00000673246294620462760FFF717FF40B1F5
:1003D000012804D0F61D26F007060836D8E7361D9A
:1003E000D6E72846DAE7206ABDE8F0812DE9F0413A
:1003F0000646002410687529314616A510D0AFF3C3
:100400000080002802DA404213A507E031688A071D
:1004100001D512A502E0490704D511A5012401E088
:10042000AFF3008000210A2206F1240709E0B0FBA7
:10043000F2FCB0FBF2F302FB1C003030785418469B
:10044000491C0028F3D123462A463046BDE8F04136
:1004500000F055B8000000002D0000002B00000047
:10046000200000004FF000020429C0F0128010F0BC
:10047000030C00F01B80CCF1040CBCF1020F18BF80
:1004800000F8012BA8BF20F8022BA1EB0C0100F013
:100490000DB85FEAC17C24BF00F8012B00F8012BE6
:1004A00048BF00F8012B70474FF0000200B513461B
:1004B00094469646203922BFA0E80C50A0E80C5084
:1004C000B1F12001BFF4F7AF090728BFA0E80C5035
:1004D00048BF0CC05DF804EB890028BF40F8042B2E
:1004E00008BF704748BF20F8022B11F0804F18BF9B
:1004F00000F8012B704770477047704770472DE92F
:10050000F0470D4699469246044600F124080168DA
:10051000880604D5E06921F01001216000E0012087
:10052000A84201DD471B00E00027A1697A1902EB10
:100530000900081AA0612078C00602D42046AFF353
:100540000080002608E0D4E901211AF8060090474F
:10055000206A401C761C20624E45F4DB2078C006E1
:100560000AD52046AFF3008006E0D4E9012130200F
:100570009047206A401C2062381EA7F10107F4DC76
:1005800007E0D4E9012118F805009047206A401CD3
:100590002062281EA5F10105F3DC2046AFF30080A0
:1005A0002078000602D50220BDE8F0870120FBE795
:1005B000074B70B50D467B4400F011F80446284601
:1005C00000F020F810B14FF0FF3070BD204670BD34
:1005D0005F27000001694A1C02610878704700B576
:1005E0008FB0CDE901310021059105497944CDE96C
:1005F000031011466846FFF7C5FE0FB000BD0000AE
:10060000E5FFFFFF007B00F080007047754600F0BB
:100610002BF8AE4605006946534620F00700854694
:1006200018B020B5FFF718FEBDE820404FF00006D7
:100630004FF000074FF000084FF0000B21F00701CA
:10064000AC46ACE8C009ACE8C009ACE8C009ACE80D
:10065000C0098D46704710B50446AFF300802046B0
:10066000BDE81040FFF7DEBD004870472C020020B7
:1006700010B53C2318221949194800F0EDFF19481C
:100680000088062829DB282000F020FB00224FF4F8
:100690000041154800F0BCFA14A0FFF767FE0024E3
:1006A00005E00E48015D14A0FFF760FE641C0D48D4
:1006B00000888442F5DD12A0FFF758FE282000F0E4
:1006C00027FB0122D103084800F0A2FA18210348B1
:1006D000FFF7C8FE00200349088010BD84010020F8
:1006E0002C0100201E000020001802400D0AE5BC6D
:1006F00080E5A78B5C720A0025640D0A00000000EB
:100700000D0AE7BB93E69D9F0D0A000000B587B078
:10071000142102A8FFF7C8FE00BF00200190564830
:10072000006840F00400544908600846006800F082
:100730000400019000BF00BF00BF002001900846E8
:10074000006840F0800008600846006800F0800003
:10075000019000BF00BF00BF002001900846006864
:1007600040F0400008600846006800F0400001903A
:1007700000BF00BF00BF002001900846006840F0A5
:10078000020008600846006800F00200019000BF07
:1007900000BF00BF002001900846006840F0010043
:1007A00008600846006800F00100019000BF00BF2B
:1007B00000BF002001900846006840F00800086073
:1007C0000846006800F00800019000BF00BF012249
:1007D0004FF4C041294800F01BFA0122D1032748F9
:1007E00000F016FA4FF400600290254803900120B3
:1007F000049002A9214800F009F94FF460400290EA
:100800000120039004900220059002A91B4800F0EB
:10081000FDF84FF4004002900120039004900590F1
:1008200002A9164800F0F2F8102002900020039070
:1008300004900220059002A9124800F0E7F84FF456
:10084000807002900E4803900120049002A90E4887
:1008500000F0DCF801220021282000F069FA2820AD
:1008600000F034FA00221146172000F061FA172038
:1008700000F02CFA07B000BD3038024000180240EA
:100880000000211000040240000C024000BFFEE7FF
:100890007047000010B50B48006800F4006078B1A4
:1008A0004FF40060074908600748006830B901202C
:1008B00005490860172000F02BFA01E0FFF7D8FE89
:1008C00010BD0000143C01400000002010B5174886
:1008D000006800F4807040B34FF4807013490860E2
:1008E0001348006802280DD100BF00BF00BF00BF41
:1008F00000BF00BF0122D1030E4800F089F9172084
:1009000000F0E4F90A48006801280ED1082001F03F
:10091000FFFC00224FF40041064800F079F9032063
:1009200001F0F6FC02200249086010BD143C0140B1
:10093000000000200018024070B50446A56D00F0CC
:1009400073F9064694F83500022808D080206065C7
:1009500000BF002084F8340000BF012070BD206873
:10096000006820F01600216808602068406920F0C7
:10097000800021684861206C08B9A06C28B120680B
:10098000006820F00800216808602068006820F0F6
:100990000100216808600FE000F046F9801B05287F
:1009A0000AD92020606500BF002084F8340000BF11
:1009B000032084F83500D1E72068006800F00100CA
:1009C0000028E9D194F85C103F208840A86000BF5F
:1009D000002084F8340000BF012084F83500002096
:1009E000BCE7014691F83500022803D08020486515
:1009F00001207047052081F835000868006820F064
:100A000001000A6810600020F3E70000F8B5024614
:100A10000B460025002400200021DEE0012606FA16
:100A200001F51E6806EA0504AC4275D11E7906F090
:100A30000306012E04D01E7906F00306022E13D100
:100A400090684F000326BE40B0434F00DE68BE40B2
:100A500030439060506801268E40B0431E79C6F343
:100A600000168E40304350601E7906F00306032EB8
:100A700009D0D0684F000326BE40B0434F009E68A7
:100A8000BE403043D0601E7906F00306022E13D11B
:100A9000CF0802F1200656F827004E07F70E0F2662
:100AA000BE40B0434F07FF0E1E69BE403043CF0823
:100AB00002F1200646F8270010684F000326BE40CA
:100AC000B0431E7906F003064F00BE40304310606D
:100AD0005E6806F08056B6F1805F7DD100BF0026CB
:100AE0000096404E366846F480463E4F3E603E4695
:100AF000366806F48046009600BF00BF3A4E8F0865
:100B000056F827008E07370F0F26BE40B043374EEA
:100B1000B24202D1002624E05EE0354EB24201D15D
:100B200001261EE0334EB24201D1022619E0324EB8
:100B3000B24201D1032614E0304EB24201D1042664
:100B40000FE02F4EB24201D105260AE02D4EB242EF
:100B500001D1062605E02C4EB24201D1072600E065
:100B600008268F073F0FBE4030431F4E8F0846F8C0
:100B70002700264E3068A0435E6806F48036B6F53E
:100B8000803F00D12043214E3060361D3068A043A5
:100B90005E6806F40036B6F5003F00D120431B4ED8
:100BA000361D3060361D3068A0435E6806F480163E
:100BB000B6F5801F00D12043144E08363060361D34
:100BC0003068A0435E6806F40016B6F5001F00D139
:100BD00020430E4E0C363060491C1029FFF41EAF26
:100BE000F8BD0000443802400838014000000240CF
:100BF0000004024000080240000C024000100240C5
:100C00000014024000180240001C0240003C014059
:100C10000AB1816101E00B048361704701480068FB
:100C2000000C7047002004E0014800687047000095
:100C3000140000200348006803490978084401496A
:100C400008607047140000201C00002010B50A48FE
:100C5000006840F40070084908600846006840F4E5
:100C600080600860032000F0A1F80F2000F006F873
:100C700000F02AF8002010BD003C024070B5044688
:100C80000E4800784FF47A71B1FBF0F00C49096816
:100C9000B1FBF0F5284600F06DFF08B1012070BDF2
:100CA000102C07D200222146501E00F041F80548C2
:100CB000046001E00120F2E70020F0E71C000020C2
:100CC00004000020180000207047000010B5014605
:100CD0000846002817DB00F01F0301229A400B4B47
:100CE000440943F8242000BF00BF00BFBFF34F8F6B
:100CF00000BF00BF00BF00BF00BF00BFBFF36F8FCA
:100D000000BF00BF00BF00BF10BD000080E100E0D9
:100D100001460846002809DB00F01F0301229A4023
:100D200043099B0003F1E023C3F8002100BF704793
:100D30002DE9F05F80460D461646002701F0C4FFFE
:100D4000074639462A46334601F00700C0F1070A34
:100D5000BAF1040F02D94FF0040A01E0C0F1070A0A
:100D6000D14600F1040ABAF1070F02D24FF0000A8F
:100D700001E0A0F1030AD4464FF0010A0AFA09FA89
:100D8000AAF1010A0AEA020A0AFA0CFA4FF0010B68
:100D90000BFA0CFBABF1010B0BEA030B4AEA0B0459
:100DA0002146404601F098FFBDE8F09F00BF00F0EB
:100DB0000702064B19684FF6FF031940044B0B431B
:100DC00043EA0221014B196000BF70470CED00E0BF
:100DD0000000FA0570B504460D460CB9012070BD3F
:100DE0005848006800F00700A84209D255490D7024
:100DF0000846006800F00700A84201D00120EEE795
:100E0000207800F0020002281DD1207800F00400B4
:100E1000042805D14C48006840F4E0504A49086075
:100E2000207800F00800082805D14748006840F401
:100E30006040454908604448006820F0F000A1681F
:100E4000084341490860207800F00100A8B36068B9
:100E5000012807D13C4808380068C0F34040B8B9C1
:100E60000120BCE76068022802D06068032807D12F
:100E7000354808380068C0F3406048B90120AEE743
:100E8000314808380068C0F3400008B90120A6E7DF
:100E90002D48006820F00300616808432A49086073
:100EA000FFF7C2FE064609E0FFF7BEFE801B41F2D7
:100EB0008831884202D9032091E707E02248006880
:100EC00000F00C006168B0EB810FEDD11D480068A7
:100ED00000F00700A84209D91A490D7008460068B9
:100EE00000F00700A84201D0012078E7207800F048
:100EF0000400042807D11448006820F4E050E16899
:100F0000084311490860207800F00800082808D13B
:100F10000D48006820F46040216940EAC1000A4998
:100F2000086000F03FF808490968C1F30311074A57
:100F3000515CC8400649086006480068FFF79EFEFD
:100F400000204CE7003C0240083802400A2F00080D
:100F500004000020180000200148006870470000CD
:100F60000400002000B5FFF7F7FF04490968C1F34A
:100F70008221034A515CC84000BD0000083802408D
:100F80001A2F000800B5FFF7E7FF04490968C1F30D
:100F90004231034A515CC84000BD0000083802409D
:100FA0001A2F00082DE9F047002400250026A1464D
:100FB0002548006800F00C0020B1042805D008285E
:100FC0003AD105E0DFF8849039E0DFF8849036E02C
:100FD0001D48001F006800F03F041B48001F006808
:100FE00000F4800078B11A481749091F0968C1F355
:100FF0008811A0FB01700146224600233846FFF706
:101000003EF905460EE011480F49091F0968C1F372
:101010008811A0FB01700146224600233846FFF7E5
:101020002EF905460848001F0068C0F30140401C27
:101030004600B5FBF6F902E0DFF8109000BF00BFF4
:101040004846BDE8F0870000083802400024F4005C
:1010500000127A00F8B504460CB90120F8BD2078DA
:1010600000F00100002874D0F948006800F00C007E
:1010700004280DD0F648006800F00C00082813D1B1
:10108000F348001F006800F48000B0F5800F0BD11A
:10109000EF4808380068C0F34040002859D0606825
:1010A000002856D10120D9E700BF6068B0F5803F25
:1010B00008D1E7480838006840F48030E44908392E
:1010C00008601EE06068B0F5A02F0DD1E048083838
:1010D000006840F48020DE4908390860084600684E
:1010E00040F4803008600CE0D9480838006820F4EB
:1010F0008030D749083908600846006820F480200D
:10110000086000BF606890B1FFF78EFD054606E0FD
:10111000FFF78AFD401B642801D903209EE7CC48D5
:1011200008380068C0F340400028F1D011E0FFF714
:101130007BFD054606E0FFF777FD401B642801D9DB
:1011400003208BE7C24808380068C0F340400028FD
:10115000F1D1207800F0020002285FD1BC4800687D
:1011600000F00C0058B1BA48006800F00C000828E4
:101170001CD1B748001F006800F48000B0B9B44823
:1011800008380068C0F3400020B1E068012801D0B1
:10119000012063E7AE480838006820F0F8002169B4
:1011A00040EAC100AA490839086037E0E06800B3A6
:1011B0000120A8490860FFF737FD054606E0FFF764
:1011C00033FD401B022801D9032047E7A048083817
:1011D0000068C0F340000028F1D09D48083800683E
:1011E00020F0F800216940EAC100994908390860F7
:1011F00014E0002097490860FFF716FD054606E059
:10120000FFF712FD401B022801D9032026E7904872
:1012100008380068C0F340000028F1D1207800F0C1
:10122000080008282CD16069A8B101208A4908600B
:10123000FFF7FAFC054606E0FFF7F6FC401B022824
:1012400001D903200AE782486C300068C0F34000EF
:101250000028F1D014E000207F490860FFF7E4FC8B
:10126000054606E0FFF7E0FC401B022801D90320F9
:10127000F4E677486C300068C0F340000028F1D1F4
:10128000207800F00400042870D10027704838301E
:10129000006800F0805090B900BF002000906C48BA
:1012A0003830006840F0805069493831086008469D
:1012B000006800F08050009000BF00BF0127674821
:1012C000006800F48070B0B96448006840F4807031
:1012D00062490860FFF7A8FC054606E0FFF7A4FC9A
:1012E000401B022801D90320B8E65C48006800F4DE
:1012F00080700028F2D000BFA068012808D15448AF
:101300006830006840F001005149683108601DE014
:10131000A06805280DD14E486830006840F00400F0
:101320004B49683108600846006840F001000860D9
:101330000CE047486830006820F0010044496831FB
:1013400008600846006820F00400086000BFA0683C
:10135000A8B1FFF769FC054609E0FFF765FC401BF3
:1013600041F28831884202D9032077E626E03848E6
:1013700068300068C0F340000028EED013E0FFF7AB
:1013800053FC054608E0FFF74FFC401B41F2883153
:10139000884201D9032061E62D4868300068C0F317
:1013A00040000028EFD1012F07D1294838300068CC
:1013B00020F0805026493831086000BFA06900281D
:1013C00045D02348006800F00C0008285DD0A069D3
:1013D000022845D100201F490866FFF725FC054675
:1013E00006E0FFF721FC401B022801D9032035E667
:1013F000174808380068C0F340600028F1D1D4E9EC
:1014000007010843616A40EA81110122A06AC2EB28
:10141000500041EA00412C20005D41EA00600C4987
:10142000091F086001200B490866FFF7FDFB054610
:1014300006E0FFF7F9FB401B022801D903200DE667
:10144000034808380068C0F340600028F1D049E044
:101450000838024000004742800E474200700040BA
:10146000002021490866FFF7DFFB054606E0FFF78D
:10147000DBFB401B022801D90320EFE51B48006875
:10148000C0F340600028F2D12CE0A069012800D10F
:10149000E4E51648001D0668A069012820D006F47E
:1014A0008001E06981421BD106F03F01206A814240
:1014B00016D147F6C0703040616AB0EB811F0FD182
:1014C00006F440310122A06AC2EB5000B1EB004F9C
:1014D00006D106F070612C20005DB1EB006F01D0E9
:1014E0000120BBE50020B9E500004742003802407A
:1014F00010B504460CB9012010BD606A38B96068A7
:10150000B0F5827F00D105E00021E16102E0002119
:1015100021616161A06AB0F5005F00D100BF94F85D
:10152000510028B9002084F85000204600F050F8FF
:10153000022084F851002068006820F040002168F3
:101540000860A08800F48270218901F404410843F6
:10155000A18901F400610843217C01F002010843E4
:10156000217D01F001010843218B01F40071084342
:10157000217F01F0380108432021095D01F080013D
:101580000843218D01F400510843216808600421BB
:10159000A06901EA104094F8241001F010010843FA
:1015A00021684860A06AB0F5005F03D1A08D80B2C9
:1015B000216808612068C06920F400602168C86162
:1015C00000206065012084F85100002094E70000AD
:1015D00010B586B00446142101A8FEF765FF1B492B
:1015E000206888422FD100BF002000901848006872
:1015F00040F48050164908600846006800F48050A6
:10160000009000BF00BF00BF0020009010481438B9
:10161000006840F002000E4914390860084600686E
:1016200000F00200009000BF00BF182001900220CF
:10163000029000200390032004900520059001A94A
:101640000448FFF7E3F906B010BD00000030014088
:1016500044380240000402402DE9FC470446884615
:1016600017461D460020019081466068B0F5827FD4
:101670000DD1A06858B9042084F851003B46424679
:1016800041462046009500F0F8F8BDE8FC8700BF11
:1016900094F85000012801D10220F6E7012084F8D7
:1016A000500000BFFFF7C0FA064694F85100012829
:1016B00002D04FF00209D6E0B8F1000F00D017B900
:1016C0004FF00109CFE0042084F85100002060654C
:1016D000C4F83880A787E7872063A086E086206467
:1016E0006064A06AB0F5005F10D100BF2068006898
:1016F00020F40050216808602068006840F4005021
:101700002168086000BFE08F401EE087A068B0F548
:10171000004F0BD12068006820F04000216808606D
:101720002068006820F48040216808602068006814
:1017300000F04000402805D02068006840F04000DC
:1017400021680860E068F8B91AE02068806800F055
:10175000010050B12068007BA16B0870A06B401C99
:10176000A063E08F401EE0870AE0FFF75DFA801B70
:10177000A84201D3681C00B915B94FF0030972E003
:10178000E08F0028E1D11EE01AE02068806800F0B8
:10179000010050B12068C068A16B0880A06B801C5C
:1017A000A063E08F401EE0870AE0FFF73DFA801B50
:1017B000A84201D3681C00B915B94FF0030952E0E3
:1017C000E08F0028E1D1A06AB0F5005F30D1206839
:1017D000006840F48050216808602B4601221146C1
:1017E0002046009600F072FE10B14FF003093AE077
:1017F000E068B0F5006F04D12068C068A16B088074
:1018000003E02068007BA16B08702B460122114683
:101810002046009600F05AFE30B1606D40F00200A4
:1018200060654FF003091EE02068C068019000BFAA
:1018300032462946204600F0C9FD08B120206065E7
:101840002068806800F01000102807D1606D40F01B
:10185000020060654FF6EF7021688860606D08B126
:101860004FF0010900BF012084F8510000BF0020A3
:1018700084F8500000BF484607E72DE9F04F85B0D7
:101880000446884691461D460E9E00200490012085
:1018900002900020019000BF94F85000012803D16D
:1018A000022005B0BDE8F08F012084F8500000BF91
:1018B000FFF7BAF9074694F851B060680390AA465A
:1018C000BBF1010F0BD00398B0F5827F04D1A06863
:1018D00010B9BBF1040F02D0022001902CE1B8F145
:1018E000000F03D0B9F1000F00D015B9012001900D
:1018F00022E194F85100042802D0052084F8510018
:1019000000206065C4F83890E587A587C4F830806A
:10191000E586A58620646064A06AB0F5005F0DD1FD
:1019200000BF2068006820F400502168086020682B
:10193000006840F400502168086000BF206800681B
:1019400000F04000402805D02068006840F04000CA
:1019500021680860E068B0F5006F56D1606810B18A
:10196000BAF1010F09D1206B00882168C860206B93
:10197000801C2063E08E401EE0863FE02068806887
:1019800000F0020002281CD1E08ED0B1029801289C
:1019900017D1206B00882168C860206B801C2063F1
:1019A000E08E401EE08600200290E08E48B9A06ADA
:1019B000B0F5005F05D12068006840F480502168D0
:1019C00008602068806800F0010068B1E08F58B1BD
:1019D0002068C068A16B0880A06B801CA063E08FAA
:1019E000401EE08701200290FFF71EF9C01BB042A5
:1019F00004D3701C10B1032001909DE0E08E0028FC
:101A0000BCD1E08F0028B9D156E0606810B1BAF1BE
:101A1000010F09D1206B007821680873206B401CEE
:101A20002063E08E401EE08640E02068806800F081
:101A3000020002281CD1E08ED0B10298012817D1F3
:101A4000206B007821680873206B401C2063E08EB7
:101A5000401EE08600200290E08E48B9A06AB0F5F2
:101A6000005F05D12068006840F48050216808605C
:101A70002068806800F0010068B1E08F58B12068EC
:101A8000C068A16B0870A06B401CA063E08F401E73
:101A9000E08701200290FFF7C7F8C01BB04201D3D6
:101AA000701C00B916B90320019045E0E08E0028B3
:101AB000BBD1E08F0028B8D1A06AB0F5005F12D189
:101AC0003346012211462046009700F0FFFC30B15A
:101AD000606D40F002006065032001902CE02068FA
:101AE000C068049000BF2068806800F010001028D3
:101AF00009D1606D40F0020060654FF6EF7021681B
:101B00008860012001903A463146204600F0A8FC4A
:101B100020B101200190202060650DE0A06850B93F
:101B200000BF002000902068C06800902068806896
:101B3000009000BF00BF00BF012084F8510000BF2B
:101B4000002084F8500000BF0198AAE6042808D1BC
:101B50004FF0E021096941F004014FF0E0221161EA
:101B600007E04FF0E021096921F004014FF0E02285
:101B70001161704770B504462546681EB0F1807F3C
:101B800001D301200FE0681E4FF0E02148610F21D2
:101B90004FF0FF3001F0A0F800204FF0E021886105
:101BA00007200861002070BD70B504460D4616463A
:101BB00000BF94F83C00012801D1022070BD012033
:101BC00084F83C0000BF36B1042E1BD0082E31D063
:101BD0000C2E5ED145E02946206800F071FD20689A
:101BE000806940F00800216888612068806920F0E1
:101BF0000400216888612068806929690843216898
:101C0000886147E02946206800F092FD20688069DD
:101C100040F40060216888612068806920F4806059
:101C20002168886120688069296940EA012021686B
:101C300088612FE02946206800F0B8FD2068C0695F
:101C400040F008002168C8612068C06920F00400E5
:101C50002168C8612068C069296908432168C86192
:101C600018E02946206800F0DDFD2068C06940F4D6
:101C700000602168C8612068C06920F48060216824
:101C8000C8612068C069296940EA01202168C861EB
:101C900000E000BF00BF00BF002084F83C0000BF90
:101CA00000BF8BE710B504460CB9012010BD94F8B5
:101CB0003D0028B9002084F83C00204600F026F8BA
:101CC000022084F83D00211D206800F07BFC0120EB
:101CD00084F8460000BF84F83E0001213F200155F2
:101CE000402001554120015500BF00BF012084F86C
:101CF000420043200155442001554520015500BFB5
:101D0000012084F83D000020D0E7000010B586B027
:101D100004462068B0F1804F34D100BF00BF0020DE
:101D200000901948006840F0010017490860084613
:101D3000006800F00100009000BF00BF00BF00BFBE
:101D400000BF0020009010481030006840F00100F3
:101D50000D49103108600846006800F0010000904D
:101D600000BF00BF00BF04200190022002900120AC
:101D70000390022004900120059001A90348FEF77A
:101D800045FE00BF06B010BD3038024000000240E2
:101D900070B504460D4615B994F83E000BE0042DCD
:101DA00002D13F20005D06E0082D02D14020005DF9
:101DB00001E04120005D012801D0012070BD1DB966
:101DC000022084F83E000EE0042D03D102213F20C2
:101DD000015508E0082D03D102214020015502E001
:101DE00002214120015501222946206800F056FCBD
:101DF00023492068884203D022492068884201D1C3
:101E0000012000E0002028B12068406C40F4004030
:101E1000216848641A49206888421BD02068B0F1C4
:101E2000804F17D018492068884213D0174920687E
:101E300088420FD01649206888420BD0114920688B
:101E4000884207D013492068884203D0124920688D
:101E500088420CD12068806800F00706062E0CD05E
:101E60002068006840F001002168086005E02068F3
:101E7000006840F001002168086000209EE7000033
:101E80000000014000040140000400400008004040
:101E9000000C0040004001400018004070477047AF
:101EA00001460022002391F83D2091F83E3042EA9D
:101EB000030070472DE9F84F044620680568206844
:101EC000C668206847694FF00009CA4605F00F0947
:101ED000B9F1000F0AD105F0200038B106F020005A
:101EE00020B1204600F0FDFCBDE8F88FB9F1000FED
:101EF00072D007F0010018B906F4907000286BD07A
:101F000005F0010030B106F4807018B1206C40F08B
:101F10000100206405F0040030B107F0010018B1A1
:101F2000206C40F00200206405F0020030B107F0A0
:101F3000010018B1206C40F00400206405F0080096
:101F400048B106F0200010B907F0010018B1206C6C
:101F500040F008002064206C70B305F0200028B128
:101F600006F0200010B1204600F0BBFC206840695C
:101F7000C0F3801A206C00F0080010B9BAF1000F0D
:101F800023D0204600F082FC2068406900F0400029
:101F9000402816D12068406920F04000216848613F
:101FA000A06B50B15648A16B0865A06BFEF719FDF8
:101FB00010B1A06B016D88470CE02046FFF76FFF62
:101FC00008E02046FFF76BFF04E02046FFF767FFBD
:101FD0000020206488E7FFE7206B012879D105F015
:101FE0001000002875D006F01000002871D000BF46
:101FF00000200090206800680090206840680090F1
:1020000000BF00BF2068406900F04000402839D17F
:10201000A06B006840681FFA80F8B8F1000F30D05C
:10202000A08D40452DDDA4F82E80A06BC069B0F5D1
:10203000807F1FD02068C06820F480702168C8604D
:102040002068406920F001002168486120684069EB
:1020500020F0400021684861202084F83E000020E4
:1020600020632068C06820F010002168C860A06B61
:10207000FEF762FCA08DE28D801A81B22046FFF748
:102080000DFF31E7A08DE18D401A1FFA80F8E08D39
:10209000E8B1B8F1000F1AD02068C06820F4907041
:1020A0002168C8602068406920F00100216848610B
:1020B000202084F83E00002020632068C06820F0C3
:1020C00010002168C86041462046FFF7E7FE0BE795
:1020D000FFE705F0800030B106F0800018B120461F
:1020E00000F097FD00E705F0400030B106F0400039
:1020F00018B1204600F0E5FBF6E600BFF4E600006C
:102100007928000810B504460CB9012010BDA0695B
:1021100000B100E000BF94F83D0028B9002084F829
:102120003C00204600F028F8242084F83D00206878
:10213000C06820F400502168C860204600F030FCE0
:102140002068006920F49040216808612068406997
:1021500020F02A00216848612068C06840F40050DF
:102160002168C86000202064202084F83D0084F8A5
:102170003E000020CAE7000010B586B004462D4995
:102180002068884254D100BF00BF002000902A4838
:10219000006840F01000284908600846006800F018
:1021A0001000009000BF00BF00BF00BF00BF0020B4
:1021B000009021481438006840F002001E4914398C
:1021C00008600846006800F00200009000BF00BFF1
:1021D00000BF00BF00BF002000900846006840F02C
:1021E000020008600846006800F00200009000BF8E
:1021F00000BF00BF40200190022002900120039008
:10220000022004900720059001A90C48FEF7FEFB70
:10221000802001900720059001A90848FEF7F6FBF1
:102220002520FEF775FD032211462520FEF780FDCF
:1022300006B010BD001001404438024000040240C6
:1022400070B504460D46164694F83E00202816D177
:1022500005B10EB9012070BD00BF94F83C00012803
:1022600001D10220F7E7012084F83C0000BF0020E4
:10227000206332462946204600F0A8FCEBE7022006
:10228000E9E700001D4A0168914236D11C490988DE
:1022900001F4004189BB1A49098801F4804171B1F8
:1022A000184909780A2903D00021154A118024E031
:1022B0001349098841F40041114A11801DE0114978
:1022C00009780D2906D10E49098841F480410C4A4C
:1022D000118012E00B490978094A1288C2F30D02F5
:1022E000094B995406490988491C054A1180114631
:1022F0000988C72901DD00211180704700100140C5
:102300001000002012000020200000207047000074
:1023100011B526E0009CB4F5617F02D94FF46174D9
:1023200000E0009C23464FF0E024A069A82404FBB1
:102330001301002908DB00BF4FF0E024A2698242AC
:102340000CDA8A42F8DA09E0084C214400BF4FF069
:10235000E024A2698242FADD8A42F8DC009CE41A99
:102360000094009C002CD5D118BD000040900200C4
:1023700000BFFEE710B51148114908604FF48270A4
:10238000486000210E488160C160016141614FF4E5
:10239000007181613821C161002101624162816265
:1023A0000A21C162FFF7A4F805480068006840F000
:1023B000400003490968086010BD0000003001407A
:1023C0002C01002000BFFEE770477047F8B50446B7
:1023D0000E4615466068B0F5827F0DD1A068B0F555
:1023E000004F03D0A068B0F5806F05D12068006869
:1023F00020F04000216808606068B0F5827F1FD13E
:10240000A068B0F5806F0DD03346002280212046B1
:10241000009500F05BF808B3606D40F02000606547
:102420000320F8BD3346002201212046009500F02C
:102430004DF898B1606D40F0200060650320F0E732
:102440003346002201212046009500F03FF828B1D4
:10245000606D40F0200060650320E2E70020E0E7C7
:102460007CB504460D461646164800681821B0FB98
:10247000F1F01549B0FBF1F04FF47A714843019047
:102480006068B0F5827F0DD12B4600228021204666
:10249000009600F01BF898B1606D40F02000606578
:1024A00003207CBD00BF019800B908E00198401EE0
:1024B000019020688068C0F3C0100028F3D100BFED
:1024C0000020EEE70400002040420F002DE9F84F05
:1024D00004460D4690461E46DDF82890FEF7A4FB04
:1024E000A0EB0900371AFEF79FFB82462C480068D4
:1024F000C0F3CB307843009045E0701C002842D0F8
:10250000FEF792FBA0EB0A00B84200D2A7BB2068FE
:10251000406820F0E000216848606068B0F5827F84
:102520000DD1A068B0F5004F03D0A068B0F5806F62
:1025300005D12068006820F0400021680860A06A8A
:10254000B0F5005F0DD100BF2068006820F4005096
:10255000216808602068006840F400502168086025
:1025600000BF012084F8510000BF002084F8500013
:1025700000BF0320BDE8F88FFFE7009800B90027EF
:102580000098401E0090206880682840A84201D131
:10259000012000E000204045AFD10020EAE7000024
:1025A00004000020704710B5FEF744FB10BD00008A
:1025B0000348006840F4700001490860704700005B
:1025C00088ED00E010B50268294B98420ED0B0F1BA
:1025D000804F0BD0274B984208D0274B984205D00C
:1025E000264B984202D0264B984203D122F070022B
:1025F0004B681A431E4B984220D0B0F1804F1DD03B
:102600001C4B98421AD01C4B984217D01B4B984237
:1026100014D01B4B984211D01A4B98420ED01A4B33
:1026200098420BD0194B984208D0194B984205D0CC
:10263000184B984202D0184B984203D122F44072B2
:10264000CB681A4322F080034C6943EA040202601B
:102650008B68C3620B688362054B984202D0084BBB
:10266000984201D10B6903630123436110BD00004F
:10267000000001400004004000080040000C004041
:102680000004014000400140004401400048014076
:1026900000180040001C00400020004030B501F050
:1026A0001F05012404FA05F3046A9C430462046ACA
:1026B00001F01F0502FA05F52C43046230BD00004D
:1026C00030B5056A25F001050562026A4368846930
:1026D00024F0700424F003040D682C4322F002025D
:1026E0008D682A43104DA84200D103E00F4DA84247
:1026F00006D100BF22F00802CD682A4322F004026E
:10270000094DA84202D0094DA84207D123F4807395
:1027100023F400734D692B438D692B43436084611F
:102720004D684563026230BD000001400004014075
:1027300030B5056A25F010050562026A43688469B0
:1027400024F4E04424F440740D6844EA052422F0A3
:1027500020028D6842EA0512124DA84200D103E022
:10276000114DA84207D100BF22F08002CD6842EA95
:10277000051222F040020B4DA84202D00A4DA84299
:1027800009D123F4806323F400634D6943EA850390
:102790008D6943EA8503436084614D688563026205
:1027A00030BD0000000001400004014030B5056A62
:1027B00025F480750562026A4368C46924F07004D8
:1027C00024F003040D682C4322F400728D6842EA61
:1027D0000522124DA84200D103E0114DA84207D1B5
:1027E00000BF22F40062CD6842EA052222F4806232
:1027F0000A4DA84202D00A4DA84209D123F48053C1
:1028000023F400534D6943EA05138D6943EA051328
:102810004360C4614D68C563026230BD0000014081
:102820000004014030B5056A25F480550562036A4D
:102830004468C26922F4E04222F440720D6842EA20
:10284000052223F400538D6843EA0533084DA8425E
:1028500002D0084DA84204D124F480444D6944EAD2
:1028600085144460C2614D680564036230BD000098
:10287000000001400004014070B50546AC6B00202B
:10288000E085E0842046FFF70AFB70BD0168C96857
:1028900021F490710268D1600168496921F0010159
:1028A00002685161016B012905D10168C96821F0F5
:1028B00010010268D160202180F83E1000210163E0
:1028C000704710B504462068C06820F040002168B9
:1028D000C860202084F83D002046FFF717FD002047
:1028E00010BD70B5044694F83E00222856D1A06869
:1028F000B0F5805F0CD1206950B90025A66A206828
:102900004068C0F308003080A06A801CA06215E017
:10291000A56A0026A068B0F5805F03D0A06828B93A
:10292000206918B920684068287004E02068406871
:1029300000F07F002870A06A401CA062E08D401E5D
:1029400080B2E08540BB2068C06820F0200021688C
:10295000C8602068C06820F480702168C860206862
:10296000406920F0010021684861202084F83E0081
:10297000206B01280AD12068C06820F0100021686F
:10298000C860A18D2046FFF789FA02E02046FFF7D4
:1029900079FC0020206370BD0020FCE70220FAE7EC
:1029A0002DE9F84F04462068006920F44050E168A2
:1029B0000843216808612169A068084361690843E8
:1029C000E169084300902068C06849F20C618843BF
:1029D000009908432168C8602068406920F440706D
:1029E000A16908432168486176492068884203D07C
:1029F00075492068884203D1FEF7C4FA814602E097
:102A0000FEF7B0FA8146E069B0F5004F6CD10220C4
:102A10006168A0FB015003461920A9FB0070014624
:102A20002A463846FDF72BFC6421B0FBF1F04FEA53
:102A3000001A02206168A0FB01510B461920A9FB76
:102A400000712A463846FDF71AFC83460220616869
:102A5000A0FB015003461920A9FB00712A46384605
:102A6000FDF70DFC6421B0FBF1F000EBC00101EBC0
:102A70000010ABEB8000322101EBC0006421B0FB01
:102A8000F1F000F0F8000AEB400A02206168A0FBB8
:102A9000015003461920A9FB007001462A4638461A
:102AA000FDF7EDFB834602206168A0FB0150034661
:102AB0001920A9FB00712A463846FDF7E0FB642186
:102AC000B0FBF1F000EBC00101EB0010ABEB8000BC
:102AD000322101EBC0006421B0FBF1F000F00700EF
:102AE0005044216888606AE004206168A0FB0150BE
:102AF00003461920A9FB007001462A463846FDF717
:102B0000BEFB824604206168A0FB015003461920E9
:102B1000A9FB007001462A463846FDF7B0FB642148
:102B2000B0FBF1F000EBC00101EB0010AAEB80005C
:102B3000322101EB00106421B0FBF1F000F0F00A4B
:102B400004206168A0FB017003461920A9FB005115
:102B50003A462846FDF793FB6421B0FBF1F00AEBFF
:102B6000001A04206168A0FB01510B461920A9FB43
:102B700000712A463846FDF782FB834604206168CF
:102B8000A0FB015003461920A9FB007001462A460C
:102B90003846FDF774FB6421B0FBF1F000EBC00197
:102BA00001EB0010ABEB8000322101EB001064213F
:102BB000B0FBF1F000F00F00504421688860BDE8E0
:102BC000F88F0000001001400014014010B50346CA
:102BD00099629A85DA8500201864222083F83E00E5
:102BE00000BF002083F83C0000BF1868C06840F4B4
:102BF00080701C68E0601868406940F001001C6843
:102C000060611868C06840F020001C68E060002027
:102C100010BD014691F83D00212828D18868B0F503
:102C2000805F0BD1086948B90A6A1088C0F30800B0
:102C30000B685860086A801C086205E00B6A581C23
:102C4000086218780B685860C88C401E80B2C8842F
:102C500058B90868C06820F080000B68D860086820
:102C6000C06840F040000B68D86000207047022028
:102C7000FCE7000070B500240F4D1048FFF71AF96B
:102C800000BF03E0641CAC4200D904E00B48FFF72E
:102C900007F92028F6D100BF002403E0641CAC42F1
:102CA00000D906E0012206490448FFF7C9FA0028C6
:102CB000F4D100BF70BD0000FFFF0100E80000205C
:102CC0001200002000BFFEE702480068C0F30220A7
:102CD000704700000CED00E010B5002804DB0A0787
:102CE000130E054A135406E00A07140E034A00F0B7
:102CF0000F031B1FD45410BD00E400E018ED00E0EA
:102D000000BF704710B504460420FEF71FFF0148BE
:102D1000046010BD0800002000BF054A126802F0E0
:102D20004002002AF9D0C2B2014B5A60704700003D
:102D30000010014030B587B004460D461C2168469E
:102D4000FDF7B2FB4FF080400E4908600846456031
:102D500000218160C460FEF7A5FF6020009020463E
:102D600004EBD071491001910220029008226946BB
:102D70000448FEF719FF08210248FFF709F807B0D9
:102D800030BD0000E4010020FDF760FF07230222B0
:102D900008214FF4A87000F029F8A820FFF7B2FF2F
:102DA0004FF4E13000F090F8FFF7E4FAFDF7AEFCE5
:102DB00009211420FFF7BEFF05A0FDF7D7FA282050
:102DC000FDF7A6FF02A0FDF7D1FA00BFFEE7000065
:102DD0000D0AE682A8E58F91E98081E79A84E6B63C
:102DE00088E681AFE4B8BA3A0D0A00002DE9F04157
:102DF00092B080460C4615461E460027302106A894
:102E0000FDF752FB142101A8FDF74EFB00BF002087
:102E100000902A48006840F0805028490860084621
:102E2000006800F08050009000BF00BF00BF00208D
:102E300000902348006840F480402149086008461B
:102E4000006800F48040009000BF00BF01200690A1
:102E50000004079002200C9041050D91CDF83C80B4
:102E60000E941095119606A8FEF7F4F807461FB1C8
:102E7000012012B0BDE8F0810F20019002200290E5
:102E8000002003904FF4A05004904FF48050059020
:102E9000052101A8FDF79EFF07460FB10120E8E7D5
:102EA000FDF7BCFE41F20101884205D105480068EA
:102EB00040F48070034908600020DAE7403802409F
:102EC00000700040003C024010B5044609480A4921
:102ED00008600846446000218160C1600161816131
:102EE0000C214161FFF70EF9012204490248FFF766
:102EF000A7F910BD00100140E800002012000020DA
:102F00004FF04070E1EE100A704700000000000032
:102F10000000010203040607080900000000010286
:102F200003040000442F00080000002020000000DF
:102F3000C4010008642F0008200000207006000073
:102F4000E0010008000000000024F4000000000080
:102F50000000000000000000000000001000000061
:042F6000010000006C
:040000050800018965
:00000001FF
